:1000000000308A005F2900000A108A100A11820756
:1000100028340C34013406340A108A100A1182077D
:10002000413468346F346A3400341C308400000872
:100030000319292801308D008C018C0B1D288D0B94
:100040001C284A308C008C0B232800000000800BF9
:100050001A2800340608C339A300220D8C008C0D29
:10006000FC308C050C083C392304860006148316EA
:100070000610000083120610831606108312003447
:10008000A008031D4528861046288614831686106E
:100090008312A10E2108A2002A20A10E2108A2008D
:1000A0002A200D308C008C0B5328003414309C0017
:1000B0001520C3308316860583128610831686109A
:1000C0008312061083160610831299011908023C48
:1000D000031C722802309C0015200330A2002A2045
:1000E000990A66280D308C008C0B74280230A2000F
:1000F0002A200D308C008C0B7B2899011908023CBA
:10010000031C8E28190804209A00A0011A08A100D7
:10011000402002309C001520990A7E286329013076
:100120001C029E001D08023C031D982840309E07BB
:100130001E0880389F00A0011F08A1004020003445
:100140001B088C000C300C020319B3280A300C0277
:100150000319BB280D300C020319C12808300C020A
:100160000319C628CB28A0010130A100402002308D
:100170009C001520D72801309C0002309D008F2064
:10018000D72801309C009D008F20D728A001103077
:10019000A1004020D7281B081F3C031CD128073092
:1001A0009B050130A0001B08A1004020D728003487
:1001B0009B0108309A009A080319EC2883168515CC
:1001C0008312851DE52808309A0029308C008C0B9D
:1001D000E72800009A03DB2883168515831285190A
:1001E000F72829308C008C0BF3280000EC282930EC
:1001F0008C008C0BF92800009A011A08033C031CA0
:100200001129A6308C008C0B0329000003109B0CD5
:1002100083168515831285190F2908309B079A0AC2
:10022000FD28190884001B08800001308D0000346F
:100230001C088D011B02031820291B088C002C2987
:100240008C0108309D009B0D8C0D1C080C020318BE
:100250008C008D0D9D0B232900340D0819089B007F
:1002600064309C0018210C0899000D083030031DE3
:1002700040291A189A159A1946291A1A2030422923
:100280009A111A128D070D089B00A02019089B00D7
:100290000A309C0018210C0899000D083030031D0D
:1002A00055299A1959291A1A20308D070D089B00D3
:1002B000A0203030990719089B00A0200034840149
:1002C0001F308305562805309C0015209901190818
:1002D0000C20990A9B00A02004301902031D6729F5
:1002E00003309A002E309B00A0209A0B7229043014
:1002F0009900FA309C001520990B79298F01900103
:1003000091019201970198010430960096011330F3
:100310009900D8208D08031D8E29862913080F3CCB
:1003200003199429970A862913309900D8208D083B
:10033000031D9B29862914309900D8208D08031DA0
:10034000A229862915309900D8208D08031DA929D6
:100350008629150814020319AF29980A8629013045
:100360001302FD3E0318C029033E622A14088F00C1
:10037000910AC02914089000920AC029970AC0293E
:1003800001309C009D008F2058309B00A0203A3007
:100390009B00A02020309B00A0200F08990018305F
:1003A0009A002D2120309B00A020110899001830C0
:1003B0009A002D2120309B00A020170899001830AA
:1003C0009A002D210530990020309B00A020990B28
:1003D000E42901309C0002309D008F2059309B00A1
:1003E000A0203A309B00A02020309B00A0201008C5
:1003F000990018309A002D2120309B00A02012086F
:10040000990018309A002D2120309B00A020180858
:10041000990018309A002D210530990020309B005A
:10042000A020990B0E2A83160510831205140130A3
:100430009C0015200F08930013089303003A03193A
:100440002B2A15308C008C0B232A00009308031DE7
:100450002A2A00301C2A83160510831205108316E1
:1004600085108312851401309C001520100893001C
:1004700013089303003A0319472A15308C008C0B9C
:100480003F2A00009308031D462A0030382A8316AD
:100490008510831285100F081E3C8D0010080D0278
:1004A000930013089303003A0319602A15308C0057
:1004B0008C0B582A00009308031D5F2A0030512A34
:1004C000822963000A108A140A118207B629BA2900
:0204D000BE2943
:02400E00F13F80
:00000001FF
